:20000000856203688E03FFB638067F1000BDFA9286FEB72815CE1A1AFF280E861DB72810F1
:20002000B7280ABDFA6A4D2B05F638072003F63808160D56565656F7280B8A10B7280CB6CB
:200040000800BDFBEFB60801B60802B60803B60806B60809B6080EB6080F20C70FB6080ECB
:20006000B6380786555FCEFFFF0843A7008C03FF26F7CEFFFF0843A100263A8C03FF26F527
:20008000C10127045C4320DE8EF7FFCE000032A700088C040026F78EF7FFCE000032A100D1
:2000A0002613088C040026F5CE00006F00088C040026F82023B63804B63808CEFAAD8E280B
:2000C00000A600363131088CFAD026F58601B728118680B7281B208B8E03FFBDF8E20E3ED4
:2000E00020FCB6380A965A8A80975A96592A0CBDFA04BDF9BDBDCB5F7EF990B60807B6380D
:2001000004B63805BDFA04D65AC560272DC5402624BDFAF3BDFB1EBDF9BD96532A09BDF970
:20012000A8BDFA92BDFC9F9653482A05BDD822205F8D75205BBDF9BD205686FFB70808B678
:2001400008057F0045BDFAF3BDFB1EBDFC1596532A03BDAC1D9653482B128D6196532A086D
:200160008D46BDFA929DFC9F8D3E20248601B710007F0049BDDEF686FF97499645842397F7
:200180004596532A088D21BDFA92BDFC9FBDD8224F979E97A1975A97468608975496532AE3
:2001A00003BDADEDBDF2E5394FCE0000F608002B0B088C8AAC26F54C810226ED39860397A7
:2001C000239727CE5707DFC2DFC6CE7070DF2BDF37863097228601970D9717CE0125DF1EC5
:2001E000860C970C8608970197049702970386029700861397408601973CBDD28E96458471
:200200003F974539964536965A36967236967B36968236968036968136967836967736D68A
:200220007F4FCE010FA7000926FBA700D77F3297773297783297813297803297823284012E
:20024000977B32977232975A32974586FF974997858630970B5FB608099753482A09482B49
:2002600004C6322002C699D748395F375CF70808B6080426095832250F8B103620EFC60853
:200280005A4824FC321B200286FF979FC6FFF7080839BDFC0825159F5BCEFAAD8E2800A6A7
:2002A00000363131088CFAD026F59E5B391F1F1F1F1F1F1F1F1F1F1F1F1FFF1F1F1FFFFF0E
:2002C000FF00FF0000FFFFFF00FFFFFFFF0200FF0A0A0A0A0A0A0A0A0A0A0A0A0A000A0A90
:2002E0000AAA00FFFF00FFE40090FC8000000000018000965A2B08BDFC082521BDD9A39FDA
:200300005BCEFAD08E2800A600363131088CFAF326F59E5B965A2B05BDFC3A24E239D65ADF
:200320002B0DBDFC082508BDF41586DDBDF637CEFFFFDF5DFEF800DF5FC609B6F8029761D1
:20034000CEF8008D39CEF0008D34CEE8008D2FCEE0008D2ACED8008D25CED0008D20CEC882
:20036000008D1BCEC0008D16CEB8008D1196532A0CCEAFFFDF5DC610CEA8008D0139DF5B5C
:20038000EE009C5F263286999B601997608699995F19975FDE5BA6029161261C4FDE5D7DB0
:2003A00008002B11AB009C5B27030920F21126085A09DF5D39313139313137D65A2B09BDA6
:2003C000FC082404337EFB2FBDFA9232C61DF72806F7280916CA100D46444444B72807F77F
:2003E00028088602B728118680B7281B7EFB2FC61DF72800F72809CE28011658078411A7DB
:2004000000088C280926F439D6452A05D67F582B020C390D39BDFA6A4D2B1EBDFA92BDFA5E
:200420006A4D2B0CBDF63786039787BDF1CA20EEB608057F0087BDFAF339BDC377251CB61D
:2004400008032611B6080285602718967F482A05B6380A200E965984DF200496598A20971E
:20046000590D390C39D67F582A0CD6452B0B582B05D67B542503BDF2E539D67F582A17D67E
:2004800045C47FD74536BDFA92967F43B728227F282032BDF4159645843F8A80974539D68E
:2004A0005A2B0EBDFC0824037EFD59BDD9A3BDF415C61DF72800F72806F7280996532B0D7E
:2004C000861DBDFD5ABDFC3A24FB7EFD59967F482A0896728520272D20528604B720037F9A
:2004E0002003B62004843F917227E99772852027078620B7200220347F2002C640F72004B8
:20050000841FB72004365F810A2D06800ACB1020F61BBDF63732CE2805472504C6102002F5
:20052000C611E700098C280026EF2007861A8D2A4F2005B620018460F62002C40C1BD67F26
:20054000C4901B977F43B72822965A2B0CBDFC3A2507967F482BF6208139B72801B7280273
:20056000B72803B72804B72805B72807B7280839BDD9A3BDF4154F43B7100036BDFC3A3219
:2005800024F58601B71000395FD758D767D7739659852027049668200ED79BD79D96904866
:2005A0004848489B9197685FCEFF4B0808088CFFF327228CFF9F260153A10026EE5D270DF8
:2005C00036BDFC3A32251BD659C4DFD759EE01D645AD0020058647BDC428BDFC082503BD86
:2005E000F2E539CA012028C4FECA022002C4FCD745967F2B03BDBCEA39B6380739B6380849
:2006000039C4FB200ACA042006C4F72002CA08D74539BDFC0825149770860897547F00A027
:20062000960C2A07847F970CBDCD4B39BDFEC7B608099753BDFBEFBDFC3A24F339BDFEC794
:20064000FEB800DF5B86999B5C19368699995B1936CE28018622BDF62A32168A10B72804A2
:2006600054545454F72803CE280532BDF62A861DB72807B6F802CE2808BDF62A207A8D477C
:200680009645BDFBEF20718D3EB60801BDFBEFBDFC3A24F5398D30B60802BDFBEFBDC377B6
:2006A0002505B6080327F0398D1DB60803BDFBEFBDC37724F539BDFC08250BBDD9A3BDFAC3
:2006C00092BDFC3A24F839BDFC082507BDD9A3BDF41539313139C43F2004C43FCA40D74530
:2006E0003996532A0BB620058A80B72005BDADED398DD49678BDFBEFBDFC3A24FB398D1153
:20070000B65C00398D0BC4DF20048D05CA20D745399653482B078650BDC42820B639DE1778
:20072000DF3BDE19DF3D961B973F39DE17DF40DE19DF42961B974439BDFC0825109770BD21
:20074000D9A3BDF2E5BDFC3A24FB7F00703900FB1E01FDE302FDED03FDE705FE0106FE0575
:2007600007FE0908FE0D11FE1212FE1213FE1225FE9526FEA827C7AE41FED642FC7A43FEC4
:20078000DA44FEE150FDF951FDFD70FEFE72DAF073FF0474FF0A80FF1E81FF2B98F8042034
:2007A000DBA621FE2C22FE3D23FE7E24FE8730FEB631FAF332D80433D9C234E80435B804D9
:2007C00036D00437E00440FC9F45FEF152DB2F71D82275FD7076F77F82DC1483DC0F84DC10
:2007E0000A85DC0586FF3887FF3890F64691F72992F72E0000000000C004C004F804F85C02
:00000001FF
